 java_crw_demo

 Timestamp is 68fa8ff9 (Thu Oct 23 20:28:41 2025)

 Preferred load address is 10000000

 Start         Length     Name                   Class
 0001:00000000 000030fdH .text$mn                CODE
 0002:00000000 000000a4H .idata$5                DATA
 0002:000000a4 00000008H .00cfg                  DATA
 0002:000000ac 00000004H .CRT$XCA                DATA
 0002:000000b0 00000004H .CRT$XCZ                DATA
 0002:000000b4 00000004H .CRT$XIA                DATA
 0002:000000b8 00000004H .CRT$XIZ                DATA
 0002:000000bc 00000004H .CRT$XPA                DATA
 0002:000000c0 00000004H .CRT$XPZ                DATA
 0002:000000c4 00000004H .CRT$XTA                DATA
 0002:000000c8 00000008H .CRT$XTZ                DATA
 0002:000000cc 00000000H .gfids$y                DATA
 0002:000000d0 000004b0H .rdata                  DATA
 0002:00000580 00000000H .rdata$CastGuardVftablesA DATA
 0002:00000580 00000000H .rdata$CastGuardVftablesC DATA
 0002:00000580 00000004H .rdata$sxdata           DATA
 0002:00000584 0000005cH .rdata$voltmd           DATA
 0002:000005e0 000002f8H .rdata$zzzdbg           DATA
 0002:000008d8 00000004H .rtc$IAA                DATA
 0002:000008dc 00000004H .rtc$IZZ                DATA
 0002:000008e0 00000004H .rtc$TAA                DATA
 0002:000008e4 00000004H .rtc$TZZ                DATA
 0002:000008e8 00000088H .xdata$x                DATA
 0002:00000970 0000007cH .edata                  DATA
 0002:000009ec 00000078H .idata$2                DATA
 0002:00000a64 00000014H .idata$3                DATA
 0002:00000a78 000000a4H .idata$4                DATA
 0002:00000b1c 00000352H .idata$6                DATA
 0003:00000000 000000e8H .data                   DATA
 0003:000000e8 00000374H .bss                    DATA
 0004:00000000 00000060H .rsrc$01                DATA
 0004:00000060 00000350H .rsrc$02                DATA

  Address         Publics by Value              Rva+Base       Lib:Object

 0000:00000000       ___AbsoluteZero            00000000     <absolute>
 0000:00000000       ___arm64x_extra_rfe_table  00000000     <absolute>
 0000:00000000       ___arm64x_extra_rfe_table_size 00000000     <absolute>
 0000:00000000       ___arm64x_native_entrypoint 00000000     <absolute>
 0000:00000000       ___arm64x_redirection_metadata 00000000     <absolute>
 0000:00000000       ___arm64x_redirection_metadata_count 00000000     <absolute>
 0000:00000000       ___dynamic_value_reloc_table 00000000     <absolute>
 0000:00000000       ___enclave_config          00000000     <absolute>
 0000:00000000       ___guard_check_icall_a64n_fptr 00000000     <absolute>
 0000:00000000       ___guard_eh_cont_count     00000000     <absolute>
 0000:00000000       ___guard_eh_cont_table     00000000     <absolute>
 0000:00000000       ___guard_fids_count        00000000     <absolute>
 0000:00000000       ___guard_fids_table        00000000     <absolute>
 0000:00000000       ___guard_iat_count         00000000     <absolute>
 0000:00000000       ___guard_iat_table         00000000     <absolute>
 0000:00000000       ___guard_longjmp_count     00000000     <absolute>
 0000:00000000       ___guard_longjmp_table     00000000     <absolute>
 0000:00000000       ___hybrid_auxiliary_delayload_iat 00000000     <absolute>
 0000:00000000       ___hybrid_auxiliary_delayload_iat_copy 00000000     <absolute>
 0000:00000000       ___hybrid_auxiliary_iat    00000000     <absolute>
 0000:00000000       ___hybrid_auxiliary_iat_copy 00000000     <absolute>
 0000:00000000       ___hybrid_code_map         00000000     <absolute>
 0000:00000000       ___hybrid_code_map_count   00000000     <absolute>
 0000:00000000       ___hybrid_image_info_bitfield 00000000     <absolute>
 0000:00000000       ___x64_code_ranges_to_entry_points 00000000     <absolute>
 0000:00000000       ___x64_code_ranges_to_entry_points_count 00000000     <absolute>
 0000:00000001       ___safe_se_handler_count   00000001     <absolute>
 0000:00000100       ___guard_flags             00000100     <absolute>
 0000:00000000       ___ImageBase               10000000     <linker-defined>
 0001:00000000       ___local_stdio_printf_options 10001000 f i java_crw_demo.obj
 0001:00000006       __snprintf_s               10001006 f i java_crw_demo.obj
 0001:00000025       __vfprintf_l               10001025 f i java_crw_demo.obj
 0001:00000049       __vsnprintf_s_l            10001049 f i java_crw_demo.obj
 0001:00000a2a       _fprintf                   10001a2a f i java_crw_demo.obj
 0001:00000e0f       _java_crw_demo@76          10001e0f f   java_crw_demo.obj
 0001:000011c5       _java_crw_demo_classname@12 100021c5 f   java_crw_demo.obj
 0001:000023e8       @__security_check_cookie@4 100033e8 f   MSVCRT:secchk.obj
 0001:00002736       __DllMainCRTStartup@12     10003736 f   MSVCRT:dll_dllmain.obj
 0001:00002759       ___raise_securityfailure   10003759 f   MSVCRT:gs_report.obj
 0001:00002781       ___report_gsfailure        10003781 f   MSVCRT:gs_report.obj
 0001:000028c8       ___security_init_cookie    100038c8 f   MSVCRT:gs_support.obj
 0001:00002913       _DllMain@12                10003913 f   MSVCRT:dll_dllmain_stub.obj
 0001:00002935       ?__scrt_initialize_type_info@@YAXXZ 10003935 f   MSVCRT:tncleanup.obj
 0001:00002941       ?__scrt_uninitialize_type_info@@YAXXZ 10003941 f   MSVCRT:tncleanup.obj
 0001:0000294d       ___local_stdio_scanf_options 1000394d f i MSVCRT:default_local_stdio_options.obj
 0001:00002953       ___scrt_initialize_default_local_stdio_options 10003953 f   MSVCRT:default_local_stdio_options.obj
 0001:000029b4       ___scrt_acquire_startup_lock 100039b4 f   MSVCRT:utility.obj
 0001:000029e6       ___scrt_dllmain_after_initialize_c 100039e6 f   MSVCRT:utility.obj
 0001:00002a11       ___scrt_dllmain_before_initialize_c 10003a11 f   MSVCRT:utility.obj
 0001:00002a1f       ___scrt_dllmain_crt_thread_attach 10003a1f f   MSVCRT:utility.obj
 0001:00002a3e       ___scrt_dllmain_crt_thread_detach 10003a3e f   MSVCRT:utility.obj
 0001:00002a4b       ___scrt_dllmain_exception_filter 10003a4b f   MSVCRT:utility.obj
 0001:00002a7f       ___scrt_dllmain_uninitialize_c 10003a7f f   MSVCRT:utility.obj
 0001:00002aa2       ___scrt_dllmain_uninitialize_critical 10003aa2 f   MSVCRT:utility.obj
 0001:00002aaf       ___scrt_initialize_crt     10003aaf f   MSVCRT:utility.obj
 0001:00002ae8       ___scrt_initialize_onexit_tables 10003ae8 f   MSVCRT:utility.obj
 0001:00002b6f       ___scrt_is_nonwritable_in_current_image 10003b6f f   MSVCRT:utility.obj
 0001:00002c03       ___scrt_release_startup_lock 10003c03 f   MSVCRT:utility.obj
 0001:00002c20       ___scrt_uninitialize_crt   10003c20 f   MSVCRT:utility.obj
 0001:00002c48       ___scrt_get_dyn_tls_init_callback 10003c48 f   MSVCRT:dyn_tls_init.obj
 0001:00002c4e       ___scrt_fastfail           10003c4e f   MSVCRT:utility_desktop.obj
 0001:00002d69       __crt_debugger_hook        10003d69 f   MSVCRT:utility_desktop.obj
 0001:00002d71       __RTC_Initialize           10003d71 f   MSVCRT:initsect.obj
 0001:00002d9d       __RTC_Terminate            10003d9d f   MSVCRT:initsect.obj
 0001:00002dd0       __SEH_prolog4              10003dd0 f   MSVCRT:sehprolg4.obj
 0001:00002e15       __except_handler4          10003e15 f   MSVCRT:chandler4gs.obj
 0001:00002e44       @_guard_check_icall_nop@4  10003e44 f i MSVCRT:guard_support.obj
 0001:00002e47       ___isa_available_init      10003e47 f   MSVCRT:cpu_disp.obj
 0001:0000301b       __get_startup_argv_mode    1000401b f   MSVCRT:argv_mode.obj
 0001:0000301f       ___scrt_is_ucrt_dll_in_use 1000401f f   MSVCRT:ucrt_detection.obj
 0001:0000302b       _memcpy                    1000402b f   vcruntime:VCRUNTIME140.dll
 0001:00003031       _memset                    10004031 f   vcruntime:VCRUNTIME140.dll
 0001:00003037       ___std_type_info_destroy_list 10004037 f   vcruntime:VCRUNTIME140.dll
 0001:0000303d       __except_handler4_common   1000403d f   vcruntime:VCRUNTIME140.dll
 0001:00003043       _strcmp                    10004043 f   ucrt:api-ms-win-crt-string-l1-1-0.dll
 0001:00003049       _strlen                    10004049 f   ucrt:api-ms-win-crt-string-l1-1-0.dll
 0001:0000304f       __initterm                 1000404f f   ucrt:api-ms-win-crt-runtime-l1-1-0.dll
 0001:00003055       __initterm_e               10004055 f   ucrt:api-ms-win-crt-runtime-l1-1-0.dll
 0001:0000305b       __seh_filter_dll           1000405b f   ucrt:api-ms-win-crt-runtime-l1-1-0.dll
 0001:00003061       __configure_narrow_argv    10004061 f   ucrt:api-ms-win-crt-runtime-l1-1-0.dll
 0001:00003067       __initialize_narrow_environment 10004067 f   ucrt:api-ms-win-crt-runtime-l1-1-0.dll
 0001:0000306d       __initialize_onexit_table  1000406d f   ucrt:api-ms-win-crt-runtime-l1-1-0.dll
 0001:00003073       __execute_onexit_table     10004073 f   ucrt:api-ms-win-crt-runtime-l1-1-0.dll
 0001:00003079       __cexit                    10004079 f   ucrt:api-ms-win-crt-runtime-l1-1-0.dll
 0001:0000307f       ___acrt_initialize         1000407f f   MSVCRT:ucrt_stubs.obj
 0001:0000307f       ___acrt_thread_attach      1000407f f   MSVCRT:ucrt_stubs.obj
 0001:0000307f       ___acrt_thread_detach      1000407f f   MSVCRT:ucrt_stubs.obj
 0001:0000307f       ___acrt_uninitialize       1000407f f   MSVCRT:ucrt_stubs.obj
 0001:0000307f       ___acrt_uninitialize_critical 1000407f f   MSVCRT:ucrt_stubs.obj
 0001:0000307f       ___scrt_stub_for_acrt_initialize 1000407f f   MSVCRT:ucrt_stubs.obj
 0001:0000307f       ___scrt_stub_for_acrt_thread_attach 1000407f f   MSVCRT:ucrt_stubs.obj
 0001:0000307f       ___scrt_stub_for_acrt_thread_detach 1000407f f   MSVCRT:ucrt_stubs.obj
 0001:0000307f       ___scrt_stub_for_acrt_uninitialize 1000407f f   MSVCRT:ucrt_stubs.obj
 0001:0000307f       ___scrt_stub_for_acrt_uninitialize_critical 1000407f f   MSVCRT:ucrt_stubs.obj
 0001:0000307f       ___vcrt_initialize         1000407f f   MSVCRT:ucrt_stubs.obj
 0001:0000307f       ___vcrt_thread_attach      1000407f f   MSVCRT:ucrt_stubs.obj
 0001:0000307f       ___vcrt_thread_detach      1000407f f   MSVCRT:ucrt_stubs.obj
 0001:0000307f       ___vcrt_uninitialize       1000407f f   MSVCRT:ucrt_stubs.obj
 0001:0000307f       ___vcrt_uninitialize_critical 1000407f f   MSVCRT:ucrt_stubs.obj
 0001:00003082       ___scrt_stub_for_is_c_termination_complete 10004082 f   MSVCRT:ucrt_stubs.obj
 0001:00003082       __is_c_termination_complete 10004082 f   MSVCRT:ucrt_stubs.obj
 0001:00003085       __filter_x86_sse2_floating_point_exception 10004085 f   MSVCRT:x86_exception_filter.obj
 0001:00003085       __filter_x86_sse2_floating_point_exception_default 10004085 f   MSVCRT:x86_exception_filter.obj
 0002:00000000       __imp__UnhandledExceptionFilter@4 10005000     kernel32:KERNEL32.dll
 0002:00000004       __imp__SetUnhandledExceptionFilter@4 10005004     kernel32:KERNEL32.dll
 0002:00000008       __imp__GetCurrentProcess@0 10005008     kernel32:KERNEL32.dll
 0002:0000000c       __imp__TerminateProcess@8  1000500c     kernel32:KERNEL32.dll
 0002:00000010       __imp__IsProcessorFeaturePresent@4 10005010     kernel32:KERNEL32.dll
 0002:00000014       __imp__QueryPerformanceCounter@4 10005014     kernel32:KERNEL32.dll
 0002:00000018       __imp__GetCurrentProcessId@0 10005018     kernel32:KERNEL32.dll
 0002:0000001c       __imp__GetCurrentThreadId@0 1000501c     kernel32:KERNEL32.dll
 0002:00000020       __imp__GetSystemTimeAsFileTime@4 10005020     kernel32:KERNEL32.dll
 0002:00000024       __imp__DisableThreadLibraryCalls@4 10005024     kernel32:KERNEL32.dll
 0002:00000028       __imp__InitializeSListHead@4 10005028     kernel32:KERNEL32.dll
 0002:0000002c       __imp__IsDebuggerPresent@0 1000502c     kernel32:KERNEL32.dll
 0002:00000030       \177KERNEL32_NULL_THUNK_DATA 10005030     kernel32:KERNEL32.dll
 0002:00000034       __imp__memcpy              10005034     vcruntime:VCRUNTIME140.dll
 0002:00000038       __imp__memset              10005038     vcruntime:VCRUNTIME140.dll
 0002:0000003c       __imp____std_type_info_destroy_list 1000503c     vcruntime:VCRUNTIME140.dll
 0002:00000040       __imp___except_handler4_common 10005040     vcruntime:VCRUNTIME140.dll
 0002:00000044       \177VCRUNTIME140_NULL_THUNK_DATA 10005044     vcruntime:VCRUNTIME140.dll
 0002:00000048       __imp__realloc             10005048     ucrt:api-ms-win-crt-heap-l1-1-0.dll
 0002:0000004c       __imp__malloc              1000504c     ucrt:api-ms-win-crt-heap-l1-1-0.dll
 0002:00000050       __imp__free                10005050     ucrt:api-ms-win-crt-heap-l1-1-0.dll
 0002:00000054       __imp__calloc              10005054     ucrt:api-ms-win-crt-heap-l1-1-0.dll
 0002:00000058       \177api-ms-win-crt-heap-l1-1-0_NULL_THUNK_DATA 10005058     ucrt:api-ms-win-crt-heap-l1-1-0.dll
 0002:0000005c       __imp___cexit              1000505c     ucrt:api-ms-win-crt-runtime-l1-1-0.dll
 0002:00000060       __imp__abort               10005060     ucrt:api-ms-win-crt-runtime-l1-1-0.dll
 0002:00000064       __imp___execute_onexit_table 10005064     ucrt:api-ms-win-crt-runtime-l1-1-0.dll
 0002:00000068       __imp___initterm           10005068     ucrt:api-ms-win-crt-runtime-l1-1-0.dll
 0002:0000006c       __imp___initterm_e         1000506c     ucrt:api-ms-win-crt-runtime-l1-1-0.dll
 0002:00000070       __imp___seh_filter_dll     10005070     ucrt:api-ms-win-crt-runtime-l1-1-0.dll
 0002:00000074       __imp___configure_narrow_argv 10005074     ucrt:api-ms-win-crt-runtime-l1-1-0.dll
 0002:00000078       __imp___initialize_narrow_environment 10005078     ucrt:api-ms-win-crt-runtime-l1-1-0.dll
 0002:0000007c       __imp___initialize_onexit_table 1000507c     ucrt:api-ms-win-crt-runtime-l1-1-0.dll
 0002:00000080       \177api-ms-win-crt-runtime-l1-1-0_NULL_THUNK_DATA 10005080     ucrt:api-ms-win-crt-runtime-l1-1-0.dll
 0002:00000084       __imp____stdio_common_vfprintf 10005084     ucrt:api-ms-win-crt-stdio-l1-1-0.dll
 0002:00000088       __imp____acrt_iob_func     10005088     ucrt:api-ms-win-crt-stdio-l1-1-0.dll
 0002:0000008c       __imp____stdio_common_vsnprintf_s 1000508c     ucrt:api-ms-win-crt-stdio-l1-1-0.dll
 0002:00000090       \177api-ms-win-crt-stdio-l1-1-0_NULL_THUNK_DATA 10005090     ucrt:api-ms-win-crt-stdio-l1-1-0.dll
 0002:00000094       __imp__strlen              10005094     ucrt:api-ms-win-crt-string-l1-1-0.dll
 0002:00000098       __imp__strcmp              10005098     ucrt:api-ms-win-crt-string-l1-1-0.dll
 0002:0000009c       __imp__strncmp             1000509c     ucrt:api-ms-win-crt-string-l1-1-0.dll
 0002:000000a0       \177api-ms-win-crt-string-l1-1-0_NULL_THUNK_DATA 100050a0     ucrt:api-ms-win-crt-string-l1-1-0.dll
 0002:000000a4       ___guard_check_icall_fptr  100050a4     MSVCRT:guard_support.obj
 0002:000000a8       ___castguard_check_failure_os_handled_fptr 100050a8     MSVCRT:guard_support.obj
 0002:000000ac       ___xc_a                    100050ac     MSVCRT:initializers.obj
 0002:000000b0       ___xc_z                    100050b0     MSVCRT:initializers.obj
 0002:000000b4       ___xi_a                    100050b4     MSVCRT:initializers.obj
 0002:000000b8       ___xi_z                    100050b8     MSVCRT:initializers.obj
 0002:000000bc       ___xp_a                    100050bc     MSVCRT:initializers.obj
 0002:000000c0       ___xp_z                    100050c0     MSVCRT:initializers.obj
 0002:000000c4       ___xt_a                    100050c4     MSVCRT:initializers.obj
 0002:000000c8       ___xt_z                    100050c8     MSVCRT:initializers.obj
 0002:000000d0       ??_C@_0BB@BKCDLAKA@CRW?3?5?$CFs?5?$FL?$CFs?3?$CFd?$FN?6@ 100050d0     java_crw_demo.obj
 0002:000000e4       ??_C@_0BA@NADODIIN@java_crw_demo?4c@ 100050e4     java_crw_demo.obj
 0002:000000f4       ??_C@_0BL@LGJCEOI@Cannot?5allocate?5?$DM?$DN?50?5bytes@ 100050f4     java_crw_demo.obj
 0002:00000110       ??_C@_0BJ@DEPBLKHG@Ran?5out?5of?5malloc?5memory@ 10005110     java_crw_demo.obj
 0002:0000012c       ??_C@_0BH@KHGJEGKN@Cannot?5deallocate?5NULL@ 1000512c     java_crw_demo.obj
 0002:00000144       ??_C@_0BN@MGOIBEOL@Cannot?5reallocate?5?$DM?$DN?50?5bytes@ 10005144     java_crw_demo.obj
 0002:00000164       ??_C@_0BB@MCIAEODB@Unknown?5constant@ 10005164     java_crw_demo.obj
 0002:00000178       ??_C@_0BN@IDOLECFE@Unknown?5tag?3?5?$CFd?0?5at?5ipos?5?$CFhu@ 10005178     java_crw_demo.obj
 0002:00000198       ??_C@_0CH@FBKNDLHC@Invalid?5opcode?5supplied?5to?5wide@ 10005198     java_crw_demo.obj
 0002:000001c0       ??_C@_0CL@FOPOJEON@Invalid?5opcode?5supplied?5to?5opco@ 100051c0     java_crw_demo.obj
 0002:000001ec       ??_C@_0BC@LGJGDDGP@unexpected?5opcode@ 100051ec     java_crw_demo.obj
 0002:00000200       ??_C@_0BC@OLNAILFP@Unexpected?5opcode@ 10005200     java_crw_demo.obj
 0002:00000214       ??_C@_0BE@DPAKJLDB@Unexpected?5widening@ 10005214     java_crw_demo.obj
 0002:00000228       ??_C@_0CO@LAEHEHNL@Unknown?5frame?5type?5in?5StackMapT@ 10005228     java_crw_demo.obj
 0002:00000258       ??_C@_0BA@OCLMCFKC@LineNumberTable@ 10005258     java_crw_demo.obj
 0002:00000268       ??_C@_0BD@CPAEPILC@LocalVariableTable@ 10005268     java_crw_demo.obj
 0002:0000027c       ??_C@_0BH@NMBDNHBD@LocalVariableTypeTable@ 1000527c     java_crw_demo.obj
 0002:00000294       ??_C@_0O@HIHEEDNJ@StackMapTable@ 10005294     java_crw_demo.obj
 0002:000002a4       ??_C@_08DICECNHA@StackMap@ 100052a4     java_crw_demo.obj
 0002:000002b0       ??_C@_06FALKBLGB@?$DMinit?$DO@ 100052b0     java_crw_demo.obj
 0002:000002b8       ??_C@_08JOGLKNJI@?$DMclinit?$DO@ 100052b8     java_crw_demo.obj
 0002:000002c4       ??_C@_08LKAKBDAJ@finalize@ 100052c4     java_crw_demo.obj
 0002:000002d0       ??_C@_0O@GIDKOGNF@currentThread@ 100052d0     java_crw_demo.obj
 0002:000002e0       ??_C@_03GAEACAIP@?$CI?$CJV@ 100052e0     java_crw_demo.obj
 0002:000002e4       ??_C@_04BCJPDBDA@Code@     100052e4     java_crw_demo.obj
 0002:000002ec       ??_C@_0BG@LGAGMCFK@pnew_file_image?$DN?$DNNULL@ 100052ec     java_crw_demo.obj
 0002:00000304       ??_C@_0BE@BLEOJIHO@pnew_file_len?$DN?$DNNULL@ 10005304     java_crw_demo.obj
 0002:00000318       ??_C@_0BD@EJGEPBHM@file_image?5?$DN?$DN?5NULL@ 10005318     java_crw_demo.obj
 0002:0000032c       ??_C@_0N@NLIOAPJJ@file_len?5?$DM?50@ 1000532c     java_crw_demo.obj
 0002:0000033c       ??_C@_0BL@LIJPLLJM@system_class?5is?5not?50?5or?51@ 1000533c     java_crw_demo.obj
 0002:00000358       ??_C@_0BE@KBKPKHPI@tclass_name?5?$DN?$DN?5NULL@ 10005358     java_crw_demo.obj
 0002:0000036c       ??_C@_0CK@HCDPGGCL@tclass_sig?5is?5not?5a?5valid?5class@ 1000536c     java_crw_demo.obj
 0002:00000398       ??_C@_05MNEAHDDF@?$CIII?$CJV@ 10005398     java_crw_demo.obj
 0002:000003a0       ??_C@_0BG@HGOFKPJC@call_sig?5is?5not?5?$CIII?$CJV@ 100053a0     java_crw_demo.obj
 0002:000003b8       ??_C@_0BI@IHOOLJKF@return_sig?5is?5not?5?$CIII?$CJV@ 100053b8     java_crw_demo.obj
 0002:000003d0       ??_C@_0BG@JLFLBLJI@?$CILjava?1lang?1Object?$DL?$CJV@ 100053d0     java_crw_demo.obj
 0002:000003e8       ??_C@_0CK@CLCDOOJG@obj_init_sig?5is?5not?5?$CILjava?1lang@ 100053e8     java_crw_demo.obj
 0002:00000414       ??_C@_0CK@NNOKKDOC@newarray_sig?5is?5not?5?$CILjava?1lang@ 10005414     java_crw_demo.obj
 0002:00000440       ??_C@_0BB@NOKBFPFO@java?1lang?1Thread@ 10005440     java_crw_demo.obj
 0002:00000454       __pDefaultRawDllMain       10005454     MSVCRT:dll_dllmain.obj
 0002:00000454       __pRawDllMain              10005454     MSVCRT:dll_dllmain.obj
 0002:00000460       __load_config_used         10005460     MSVCRT:loadcfg.obj
 0002:00000580       ___safe_se_handler_table   10005580     <linker-defined>
 0002:00000584       ___volatile_metadata       10005584     <linker-defined>
 0002:000008d8       ___rtc_iaa                 100058d8     MSVCRT:initsect.obj
 0002:000008dc       ___rtc_izz                 100058dc     MSVCRT:initsect.obj
 0002:000008e0       ___rtc_taa                 100058e0     MSVCRT:initsect.obj
 0002:000008e4       ___rtc_tzz                 100058e4     MSVCRT:initsect.obj
 0002:000009ec       __IMPORT_DESCRIPTOR_KERNEL32 100059ec     kernel32:KERNEL32.dll
 0002:00000a00       __IMPORT_DESCRIPTOR_VCRUNTIME140 10005a00     vcruntime:VCRUNTIME140.dll
 0002:00000a14       __IMPORT_DESCRIPTOR_api-ms-win-crt-stdio-l1-1-0 10005a14     ucrt:api-ms-win-crt-stdio-l1-1-0.dll
 0002:00000a28       __IMPORT_DESCRIPTOR_api-ms-win-crt-heap-l1-1-0 10005a28     ucrt:api-ms-win-crt-heap-l1-1-0.dll
 0002:00000a3c       __IMPORT_DESCRIPTOR_api-ms-win-crt-runtime-l1-1-0 10005a3c     ucrt:api-ms-win-crt-runtime-l1-1-0.dll
 0002:00000a50       __IMPORT_DESCRIPTOR_api-ms-win-crt-string-l1-1-0 10005a50     ucrt:api-ms-win-crt-string-l1-1-0.dll
 0002:00000a64       __NULL_IMPORT_DESCRIPTOR   10005a64     kernel32:KERNEL32.dll
 0003:000000cc       ___security_cookie_complement 100060cc     MSVCRT:gs_cookie.obj
 0003:000000d0       ___security_cookie         100060d0     MSVCRT:gs_cookie.obj
 0003:000000d4       ___scrt_native_dllmain_reason 100060d4     MSVCRT:utility.obj
 0003:000000e0       ___isa_enabled             100060e0     MSVCRT:cpu_disp.obj
 0003:000000e4       ___scrt_ucrt_dll_is_in_use 100060e4     MSVCRT:ucrt_stubs.obj
 0003:00000410       ?__type_info_root_node@@3U__type_info_node@@A 10006410     MSVCRT:tncleanup.obj
 0003:00000418       ?_OptionsStorage@?1??__local_stdio_scanf_options@@9@4_KA 10006418     MSVCRT:default_local_stdio_options.obj
 0003:00000420       ___scrt_current_native_startup_state 10006420     MSVCRT:utility.obj
 0003:00000424       ___scrt_native_startup_lock 10006424     MSVCRT:utility.obj
 0003:00000444       ___scrt_debugger_hook_flag 10006444     MSVCRT:utility_desktop.obj
 0003:00000448       ___isa_available           10006448     MSVCRT:cpu_disp.obj
 0003:0000044c       ___favor                   1000644c     MSVCRT:cpu_disp.obj
 0003:00000450       ?_OptionsStorage@?1??__local_stdio_printf_options@@9@9 10006450     <common>
 0003:00000458       ___dyn_tls_init_callback   10006458     <common>

 entry point at        0001:00002736

 Static symbols

 0000:ffff7000       .debug$S                   10000000     java_crw_demo.exp
 0000:ffff7000       .debug$S                   10000000     vcruntime:VCRUNTIME140.dll
 0000:ffff7000       .debug$S                   10000000     vcruntime:VCRUNTIME140.dll
 0000:ffff7000       .debug$S                   10000000     vcruntime:VCRUNTIME140.dll
 0000:ffff7000       .debug$S                   10000000     vcruntime:VCRUNTIME140.dll
 0000:ffff7000       .debug$S                   10000000     vcruntime:VCRUNTIME140.dll
 0000:ffff7000       .debug$S                   10000000     vcruntime:VCRUNTIME140.dll
 0000:ffff7000       .debug$S                   10000000     ucrt:api-ms-win-crt-heap-l1-1-0.dll
 0000:ffff7000       .debug$S                   10000000     ucrt:api-ms-win-crt-heap-l1-1-0.dll
 0000:ffff7000       .debug$S                   10000000     ucrt:api-ms-win-crt-heap-l1-1-0.dll
 0000:ffff7000       .debug$S                   10000000     ucrt:api-ms-win-crt-heap-l1-1-0.dll
 0000:ffff7000       .debug$S                   10000000     ucrt:api-ms-win-crt-runtime-l1-1-0.dll
 0000:ffff7000       .debug$S                   10000000     ucrt:api-ms-win-crt-runtime-l1-1-0.dll
 0000:ffff7000       .debug$S                   10000000     ucrt:api-ms-win-crt-runtime-l1-1-0.dll
 0000:ffff7000       .debug$S                   10000000     ucrt:api-ms-win-crt-runtime-l1-1-0.dll
 0000:ffff7000       .debug$S                   10000000     ucrt:api-ms-win-crt-runtime-l1-1-0.dll
 0000:ffff7000       .debug$S                   10000000     ucrt:api-ms-win-crt-runtime-l1-1-0.dll
 0000:ffff7000       .debug$S                   10000000     ucrt:api-ms-win-crt-runtime-l1-1-0.dll
 0000:ffff7000       .debug$S                   10000000     ucrt:api-ms-win-crt-runtime-l1-1-0.dll
 0000:ffff7000       .debug$S                   10000000     ucrt:api-ms-win-crt-runtime-l1-1-0.dll
 0000:ffff7000       .debug$S                   10000000     ucrt:api-ms-win-crt-runtime-l1-1-0.dll
 0000:ffff7000       .debug$S                   10000000     ucrt:api-ms-win-crt-runtime-l1-1-0.dll
 0000:ffff7000       .debug$S                   10000000     ucrt:api-ms-win-crt-runtime-l1-1-0.dll
 0000:ffff7000       .debug$S                   10000000     ucrt:api-ms-win-crt-runtime-l1-1-0.dll
 0000:ffff7000       .debug$S                   10000000     ucrt:api-ms-win-crt-stdio-l1-1-0.dll
 0000:ffff7000       .debug$S                   10000000     ucrt:api-ms-win-crt-stdio-l1-1-0.dll
 0000:ffff7000       .debug$S                   10000000     ucrt:api-ms-win-crt-stdio-l1-1-0.dll
 0000:ffff7000       .debug$S                   10000000     ucrt:api-ms-win-crt-string-l1-1-0.dll
 0000:ffff7000       .debug$S                   10000000     ucrt:api-ms-win-crt-string-l1-1-0.dll
 0000:ffff7000       .debug$S                   10000000     ucrt:api-ms-win-crt-string-l1-1-0.dll
 0000:ffff7000       .debug$S                   10000000     kernel32:KERNEL32.dll
 0000:ffff7000       .debug$S                   10000000     kernel32:KERNEL32.dll
 0000:ffff7000       .debug$S                   10000000     kernel32:KERNEL32.dll
 0000:ffff7000       .debug$S                   10000000     kernel32:KERNEL32.dll
 0000:ffff7000       .debug$S                   10000000     kernel32:KERNEL32.dll
 0000:ffff7000       .debug$S                   10000000     kernel32:KERNEL32.dll
 0000:ffff7000       .debug$S                   10000000     kernel32:KERNEL32.dll
 0000:ffff7000       .debug$S                   10000000     kernel32:KERNEL32.dll
 0000:ffff7000       .debug$S                   10000000     kernel32:KERNEL32.dll
 0000:ffff7000       .debug$S                   10000000     kernel32:KERNEL32.dll
 0000:ffff7000       .debug$S                   10000000     kernel32:KERNEL32.dll
 0000:ffff7000       .debug$S                   10000000     kernel32:KERNEL32.dll
 0000:ffff7000       .debug$S                   10000000     kernel32:KERNEL32.dll
 0000:ffff7000       .debug$S                   10000000     kernel32:KERNEL32.dll
 0001:0000007b       _add_new_cpool_entry       1000107b f   java_crw_demo.obj
 0001:00000157       $LN18                      10001157     java_crw_demo.obj
 0001:0000016b       $LN17                      1000116b     java_crw_demo.obj
 0001:00000177       _add_new_method_cpool_entry 10001177 f   java_crw_demo.obj
 0001:000001e1       _adjust_instruction        100011e1 f   java_crw_demo.obj
 0001:00000381       $LN66                      10001381     java_crw_demo.obj
 0001:00000395       $LN65                      10001395     java_crw_demo.obj
 0001:000003c6       _adjust_map                100013c6 f   java_crw_demo.obj
 0001:000003e6       _allocate                  100013e6 f   java_crw_demo.obj
 0001:0000042b       _allocate_clean            1000142b f   java_crw_demo.obj
 0001:00000473       _attribute_match           10001473 f   java_crw_demo.obj
 0001:000004be       _before_injection_code     100014be f   java_crw_demo.obj
 0001:0000050a       _cleanup                   1000150a f   java_crw_demo.obj
 0001:000005a2       _copy                      100015a2 f   java_crw_demo.obj
 0001:000005d4       _copyU1                    100015d4 f   java_crw_demo.obj
 0001:000005f4       _copyU2                    100015f4 f   java_crw_demo.obj
 0001:00000611       _copyU4                    10001611 f   java_crw_demo.obj
 0001:0000062e       _copyUoffset               1000162e f   java_crw_demo.obj
 0001:0000064b       _copy_attributes           1000164b f   java_crw_demo.obj
 0001:00000682       _copy_verification_types   10001682 f   java_crw_demo.obj
 0001:000006c9       _cpool_setup               100016c9 f   java_crw_demo.obj
 0001:00000949       $LN46                      10001949     java_crw_demo.obj
 0001:00000961       $LN45                      10001961     java_crw_demo.obj
 0001:00000973       _duplicate                 10001973 f   java_crw_demo.obj
 0001:0000099f       _fatal_error               1000199f f   java_crw_demo.obj
 0001:000009e6       _fillin_cpool_entry        100019e6 f   java_crw_demo.obj
 0001:00000a42       _inject_bytecodes          10001a42 f   java_crw_demo.obj
 0001:00000a9c       _inject_class              10001a9c f   java_crw_demo.obj
 0001:00000bdd       _inject_for_opcode         10001bdd f   java_crw_demo.obj
 0001:00000d55       _injection_template        10001d55 f   java_crw_demo.obj
 0001:00001295       _method_init               10002295 f   java_crw_demo.obj
 0001:0000131c       _method_inject_and_write_code 1000231c f   java_crw_demo.obj
 0001:00001406       _method_term               10002406 f   java_crw_demo.obj
 0001:00001490       _method_write              10002490 f   java_crw_demo.obj
 0001:00001545       _method_write_all          10002545 f   java_crw_demo.obj
 0001:000015a1       _method_write_bytecodes    100025a1 f   java_crw_demo.obj
 0001:00001717       _method_write_code_attribute 10002717 f   java_crw_demo.obj
 0001:000017bf       _method_write_exception_table 100027bf f   java_crw_demo.obj
 0001:00001829       _opcode_length             10002829 f   java_crw_demo.obj
 0001:00001855       _push_short_constant_bytecodes 10002855 f   java_crw_demo.obj
 0001:00001890       _random_writeU4            10002890 f   java_crw_demo.obj
 0001:000018b2       _readS2                    100028b2 f   java_crw_demo.obj
 0001:000018e4       _readU2                    100028e4 f   java_crw_demo.obj
 0001:00001906       _readU4                    10002906 f   java_crw_demo.obj
 0001:00001924       _readUoffset               10002924 f   java_crw_demo.obj
 0001:00001942       _reallocate                10002942 f   java_crw_demo.obj
 0001:0000199f       _skip_method               1000299f f   java_crw_demo.obj
 0001:00001a16       _verify_opc_wide           10002a16 f   java_crw_demo.obj
 0001:00001a72       _widen                     10002a72 f   java_crw_demo.obj
 0001:00001aa9       _writeU1                   10002aa9 f   java_crw_demo.obj
 0001:00001ac4       _writeU2                   10002ac4 f   java_crw_demo.obj
 0001:00001adc       _writeU4                   10002adc f   java_crw_demo.obj
 0001:00001af4       _writeUoffset              10002af4 f   java_crw_demo.obj
 0001:00001b1e       _write_bytes               10002b1e f   java_crw_demo.obj
 0001:00001b48       _write_cldc_stackmap_table 10002b48 f   java_crw_demo.obj
 0001:00001bb8       _write_instruction         10002bb8 f   java_crw_demo.obj
 0001:00001f8c       $LN113                     10002f8c     java_crw_demo.obj
 0001:00001fa0       $LN112                     10002fa0     java_crw_demo.obj
 0001:00001fd4       $LN115                     10002fd4     java_crw_demo.obj
 0001:00002018       $LN114                     10003018     java_crw_demo.obj
 0001:00002047       _write_line_table          10003047 f   java_crw_demo.obj
 0001:00002090       _write_stackmap_table      10003090 f   java_crw_demo.obj
 0001:00002373       _write_var_table           10003373 f   java_crw_demo.obj
 0001:000023f6       ?dllmain_crt_dispatch@@YGHQAUHINSTANCE__@@KQAX@Z 100033f6 f   MSVCRT:dll_dllmain.obj
 0001:00002449       ?dllmain_crt_process_attach@@YAHQAUHINSTANCE__@@QAX@Z 10003449 f   MSVCRT:dll_dllmain.obj
 0001:00002550       ?dllmain_crt_process_detach@@YAH_N@Z 10003550 f   MSVCRT:dll_dllmain.obj
 0001:00002600       ?dllmain_dispatch@@YAHQAUHINSTANCE__@@KQAX@Z 10003600 f   MSVCRT:dll_dllmain.obj
 0001:0000270b       ?dllmain_raw@@YGHQAUHINSTANCE__@@KQAX@Z 1000370b f   MSVCRT:dll_dllmain.obj
 0001:0000287b       ___get_entropy             1000387b f   MSVCRT:gs_support.obj
 0001:00002970       ?find_pe_section@@YAPAU_IMAGE_SECTION_HEADER@@QAEI@Z 10003970 f   MSVCRT:utility.obj
 0001:00002dd0       $$000000                   10003dd0     MSVCRT:sehprolg4.obj
 0002:00000458       _GS_ExceptionPointers      10005458     MSVCRT:gs_report.obj
 0002:000008e8       __sehtable$?dllmain_crt_process_attach@@YAHQAUHINSTANCE__@@QAX@Z 100058e8     MSVCRT:dll_dllmain.obj
 0002:00000908       __sehtable$?dllmain_crt_process_detach@@YAH_N@Z 10005908     MSVCRT:dll_dllmain.obj
 0002:00000930       __sehtable$?dllmain_dispatch@@YAHQAUHINSTANCE__@@KQAX@Z 10005930     MSVCRT:dll_dllmain.obj
 0002:00000950       __sehtable$___scrt_is_nonwritable_in_current_image 10005950     MSVCRT:utility.obj
 0002:00000970       .edata                     10005970     java_crw_demo.exp
 0002:00000998       rgpv                       10005998     java_crw_demo.exp
 0002:000009a0       rgszName                   100059a0     java_crw_demo.exp
 0002:000009a8       rgwOrd                     100059a8     java_crw_demo.exp
 0002:000009ac       szName                     100059ac     java_crw_demo.exp
 0002:000009be       $N00001                    100059be     java_crw_demo.exp
 0002:000009d0       $N00002                    100059d0     java_crw_demo.exp
 0002:00000c40       .idata$6                   10005c40     kernel32:KERNEL32.dll
 0002:00000c9c       .idata$6                   10005c9c     vcruntime:VCRUNTIME140.dll
 0002:00000dea       .idata$6                   10005dea     ucrt:api-ms-win-crt-stdio-l1-1-0.dll
 0002:00000e0a       .idata$6                   10005e0a     ucrt:api-ms-win-crt-heap-l1-1-0.dll
 0002:00000e2a       .idata$6                   10005e2a     ucrt:api-ms-win-crt-runtime-l1-1-0.dll
 0002:00000e4c       .idata$6                   10005e4c     ucrt:api-ms-win-crt-string-l1-1-0.dll
 0003:00000000       ?_opcode_length@?1??opcode_length@@9@9 10006000     java_crw_demo.obj
 0003:000000e8       ?__proc_attached@@3HA      100060e8     MSVCRT:dll_dllmain.obj
 0003:000000f0       _GS_ExceptionRecord        100060f0     MSVCRT:gs_report.obj
 0003:00000140       _GS_ContextRecord          10006140     MSVCRT:gs_report.obj
 0003:00000428       ?is_initialized_as_dll@@3_NA 10006428     MSVCRT:utility.obj
 0003:00000429       ?module_local_atexit_table_initialized@@3_NA 10006429     MSVCRT:utility.obj
 0003:0000042c       ?module_local_atexit_table@@3U_onexit_table_t@@A 1000642c     MSVCRT:utility.obj
 0003:00000438       ?module_local_at_quick_exit_table@@3U_onexit_table_t@@A 10006438     MSVCRT:utility.obj
 0004:00000060       $R000000                   10007060     java_crw_demo.dll.res
